:030000000219FDE5
:03000B000200A848
:03002B0002019A35
:03005B0002034459
:0300730002032A5B
:1000800002030406080C10182030406080040608A3
:100090000C10182030406080A0C000070F1F3F05E3
:1000A000050D050305030302C2AF306308C2638573
:1000B0007C8AD2AF32C0D0C0E0206227E525600242
:1000C000E473E525F4C3334009758A00D263F57CF7
:1000D00001D4F58A758B00758D00D262D0E0D0D046
:1000E000D2AF32C3E526334009758A00D263F57C6E
:1000F00001F4F58AC262E526F4603C3068032072A0
:1001000013758B00758D00D0E0D0D0C295C294C21B
:1001100093D2AF32C295C294C293206E0D20660A6C
:100120007414D5E0FDE57EF45290758B00758D005A
:10013000D0E0D0D0D2AF32758A00D263757C00C2D5
:100140008DD262212A01C2306805206602D2950153
:10015000C2306805206602D29401C230680520666C
:1001600002D29301C2D29230680A2066077410D579
:10017000E0FDD29501C2D29130680A206607741062
:10018000D5E0FDD29401C2D290D29230680A2066A6
:10019000077410D5E0FDD29301C2C2AFC2AD53E6E1
:1001A000EFC0D0C0E0D2D3D2AFE57D6009E57A6080
:1001B00005757A0041D7757A01C2CEE52A6007201D
:1001C0007449152A410B7800790020742EE580309F
:1001D0007E01F430E70278FF53DACF207E0343DA62
:1001E00020307E0343DA10C2D8C271E580307E0130
:1001F000F430E70279FFC3E89970CB306103752AC8
:1002000018207403752A18885FD27020740DE52BAE
:100210006004152B411B43DA01C2D8207002417DD6
:10022000A85F206102C270207431C3E894F04003DB
:1002300074F0F8E8C4540F28F87984B70302415BDE
:10024000C313C3138721200802C313200A06C3C89F
:1002500098F8415B28F8500374FFF8C3E89568509C
:1002600003E568F88822E52D54066011E533C313D1
:10027000C31324062522F52250037522FF8522246C
:10028000A824C3E52495644002A8648825E5697024
:100290000241C1C3E8AA699A5003E8FAE4F9EAC343
:1002A00033FBE56BF45B29400D256AF8E56A6002D3
:1002B000156A400B41C10AC3E56A9A5002056A7883
:1002C000FF8826C26EC3E52694F84002D26EC3E5CD
:1002D0002594404002D26420CF0AD0E0D0D043E63B
:1002E00010D2AD32C2CF053AE57D6009E57B6005ED
:1002F000757B006120757B017801E52A600530740B
:1003000002152AC3E55F94014005756200612075FE
:100310006300756C00E5622401F56250037562FFAD
:10032000D0E0D0D043E610D2AD32C2AFC0D053E659
:100330007FC260759100855694855795759104D05C
:10034000D0D2AF32C2AF53E6EFC2ADC0D0C0E0C032
:10035000F0D2D3D2AFA8FBA9FCE57D6007C3E913B7
:10036000F9E813F8C2D830710261B653DACF207EB3
:100370000343DA10307E0343DA20D271E580307E09
:1003800001F420E702618D88278928A1DD53DACFA7
:10039000207E0343DA20307E0343DA10C2D8C271D4
:1003A000307402A1C97800E580307E01F430E702A4
:1003B000A1C9885FA1B153DACF207E0343DA203090
:1003C0007E0343DA10C271206102818F53DACF209D
:1003D0007E0343DA10307E0343DA20C2D8D271881C
:1003E0005A895BC3E89558F8E99559F97B007E086E
:1003F0007A00C3E8948CE994005005755E00818111
:10040000882178A2E6A8216055C3E894C8E9940041
:100410005008E4D2E4FB7A0A815CC3E89468E9946A
:10042000015008E4D2E3FB7A0F815CC3E894D0E981
:1004300094025008E4D2E2FB7A1E815CC3E894A0E7
:10044000E994055008E4D2E1FB7A3C815CC3E8946E
:1004500098E994085008E4D2E0FB7A787E00C3E87B
:10046000955CFCE9955DFD30E70AECF42401FCEDB8
:0E047000F43400FD755E00C3EC9AED9E50035F
:10047E00755E01885C895D855A58855B597802A145
:10048E00B1C3E89527F8E99528F9307C02A195309B
:10049E007B02A195307A02A18E20750281B2E9FD10
:1004AE00E8FC81D1E9C313F9E813F8307902A18E83
:1004BE00E9C313F9E813F8307802A18EE9C313FDEE
:1004CE00E813FC206126C3EC941CED9402400281DB
:1004DE00E8ED7018C3EC94C850120529C3E52994B1
:1004EE000A5002A1C9755F00D270A1C9E529600248
:1004FE0015297888E6F97400207F087896B90302EA
:10050E00789EE624FAFEE43400FFC3EC9EFCED9FD9
:10051E00FD9208B90310A2085007207609D276A1E1
:10052E0034307602C276A2085016B9030DECF424CC
:10053E0001FCEDF43400FD02054E78007900A19522
:10054E00B90315EC33FCED33FDC3EC940AFCED94CA
:10055E0000FD50047C007D00C3EC94FFED94004040
:10056E000678FF7900A195EC8575F0A4C5F0A2F789
:10057E0033F8790040030205B178FF79000205B126
:10058E00E9C313F9E813F8307C0EE9600278FFC373
:10059E00E81338F8E43400F9C3E894FFE994004016
:1005AE000278FF885FD270206102A1C9741FF455D2
:1005BE002F4BF52FC274EB7002D274752A1830745B
:1005CE0003752A0A306102A1DD20740353DAFE207E
:1005DE007403752B06D0F0D0E0D0D0D2AD43E61028
:1005EE0032790102060D790302060D790A02060D13
:1005FE00791E02060D796402060D79C802060D7881
:10060E0017E4D5E0FDD8FAD9F6227A147B780206E3
:10061E00347A107B8C0206347A0D7BB40206347A5F
:10062E000B7BC80206347902B27DE4D291D5E0FD8F
:10063E00D294D5E0FDC294D5E0FDC291D5E0FDD2B5
:10064E0095E576D5E0FDC2957496D5E0FDD9D9EA4B
:10065E00F8D5E0FDD8FBDBCED29122C37C007D0025
:10066E0075F00005F0EA33FAEB33FB50F6EB13FBB3
:10067E00EA13FAC3E9FFE8FEE89AF8E99BF9500499
:10068E00EFF9EEF8B3EC33FCED33FDD5F0DFEDF919
:10069E00ECF822E889F08A20D2D4F8A9F07B003059
:1006AE00F70B7BFFF42401F8E9F43400F9E8852018
:1006BE00F0A4ADF0F8E98520F0A4AFF0FEED2EF930
:1006CE0074003FFA7C04C3EA13FAE913F9E813F84D
:1006DE00DCF48BF030F70AE8F42401F8E9F4340086
:1006EE00F9E889F0C2D4F8A9F02222C3E54113F942
:1006FE00E54013F8C3E54598F8E54699F9500CC363
:10070E00E89480E994FF4016020730C3E8947FE92D
:10071E0094005003020730787F790002073078800A
:10072E0079FF884A894B22E54A2547F8E54B35483B
:10073E00F9854B20E4300701F43549FA30E709C357
:10074E00EA94F0401502076EC3EA940F50030207B5
:10075E006E78FF79FF7A0F02076E780079007AF0D3
:10076E00C3E5249564500AC374019524500B020707
:10077E008CE54B20E70E02078CE54B30E7068847E9
:10078E0089488A492278A4E6FAC3E54A33F8E54B4C
:10079E0033F9D1A1E930E70BC3E89480E994FF4027
:1007AE0013E1C6C3E8947FE994005002E1C6787F56
:1007BE007900E1C6788079FFE820E715C3E5239834
:1007CE00F84009C3E8940140030207ED78010207DF
:1007DE00EDE8F424012523F840030207ED78FF88A5
:1007EE004C2278A5E6FAA848A949D1A1E930E70C30
:1007FE00C3E89401E994FF4016020821C3E894FF70
:10080E00E99400500302082178FF7900020821784C
:10081E000179FFE920E715C3E54C98F84009C3E8D4
:10082E00940140030208487801020848E8F42401C4
:10083E00254CF8400302084878FF88242278FFC22E
:10084E006420693D206A12D264C3E541940A4009CE
:10085E00C3E52594405002C26479A1E76023E541C7
:0E086E00601F74FF8541F0848539F0306A0305
:10087C0075F005A4F8C5F0600278FFC3E8956750E1
:10088C0002A867886622C3E54094C8E5419400E558
:10089C006650031401A3046002F566220208AB2221
:1008AC0075E890227883E6FFE5E820ECF7A8BDA96F
:1008BC00BE0573C3E57394084052757300E9FA7969
:1008CC00A0E76044EA7007E574601B0208E6C3E821
:1008DC0095746010E5745006600C140208F2046004
:1008EC00F90208F2E574F574C39472401B7564C088
:1008FC00C394044013756480C39404400B75644026
:10090C00C39404400375640075BB0622E564F4606F
:10091C00020564E573B4070375BB1022743279A623
:10092C0087F0A4C5F0A2F733F8C3E895644002A899
:10093C00648822882488258826886722754000755B
:10094C0041F022C2AF75C820A8CCA9CDAA3A30CFAD
:10095C00010A75C824D2AFC3EA13FAE913F9E813F4
:10096C00F8AB3BAC3C883B893CC3E89BF8E99C204A
:10097C00690A547FF9306702417221CFAD3D8A3D3F
:10098C00F9EA9D547FFA600478FF79FFAE3EAF3FE1
:10099C008B3E8C3FC3EC9FFCC3E99CF542A83BA962
:1009AC003CC3E89EF8E99FF9C3E54113FBE540130E
:1009BC00FAE82AF540E93BF54150067540FF7541D0
:1009CC00FF4119AA40AB41AC40AD417E047F02C34C
:1009DC00EB940440021E1FC3EB940840021E1FC37D
:1009EC00ED13FDEC13FCDEF7C3EA9CFAEB9DFBEF79
:1009FC006009C3E913F9E813F8DFF7EA28FAEB39D1
:100A0C00FB8A408B4150067BFF8B408B41C3EB94A0
:100A1C00025002D2673069047F0341447892E6FFAA
:100A2C00C3E537948240110FC3E53794A040010F02
:100A3C00C3EF940640027F057E03E541C4540FF9D1
:100A4C00E541C454F0F8E540C4540F28F8C3E89EBF
:100A5C00FAE99400FB4009C3EA9402EB94005004B9
:100A6C007A02E4FB41BEAA40AB41EBC4FEEAC4549B
:100A7C000F4EFCC3EA9CFAEB9400FBC3E813C313C0
:100A8C00F8EA28FAEB3400FB8A408B41C3EB940262
:100A9C004002C2677803EBC4FE7B00EAC4540F4EDD
:100AAC00FAC3EA98FA4005C3940250027A0278928B
:100ABC00E6FF30600241BE855256855357D26043E3
:100ACC00E680C3E49AF8E49BF9C3E833F8E933F918
:100ADC00306702615FE8FAE9FBD3E913FDE813FC28
:100AEC0088528953C3EF94036038EF20E00DE82C53
:100AFC00F8E93DF9ECFAEDFB020B1AE828F8E939B4
:100B0C00F9C3E82402F8E93400F97AFE7BFFC3EF5D
:100B1C009403400E8A548B55884E894F8C508D51BE
:100B2C006193885489558A4E8B4F8C508D51306906
:100B3C0020C3E53394034019E542A2E713F8E555C9
:100B4C00F4240138400B20E7087554FFF42401F518
:100B5C00556193E8FAD3E813FC8852C3EF94036011
:100B6C0020EF20E007E82CF8ECFA617FE82824025B
:100B7C00F87AFEC3EF940340088A54884E8C506177
:100B8C009388548A4E8C50E56BC3335002646BF5DA
:100B9C006B306002619D753404D26043E680E52DB4
:100BAC005406601FA840A941C2AF53E67F7591005F
:100BBC00C3E498F594E499F595759104D26043E6F5
:100BCC0080D2AF22D265754400752000306B03755E
:100BDC002040020BEFD265754400752040306B034A
:100BEC00752000D2AF7801206722E52D54066002F3
:100BFC00C265C3E54194054013780294054008781A
:100C0C0003940540027806306902780A206019E5E1
:100C1C0044601530690AC3E53394034003D53406A8
:100C2C00D2AFD26C81D171A5D2AF0000C2AF206718
:100C3C002AE541C3FB940F40027B0FEB2405307374
:100C4C000123306A02742820620123F93069027989
:100C5C0082E58D13E58B13C39940B10544E59B5494
:0E0C6C0040B5200281BB30690A08C3E8940A33
:100C7A00400108811820650261EFC26553E67F755D
:100C8A0091003067107594007595FC759104D260D7
:100C9A0043E68061EFAE40AF41C3EE33FEEF33FF70
:100CAA0050047EFF7FFFC3E49EF594E49FF595818F
:100CBA0095C3E5339402500261EF30650261EFD8C3
:100CCA000281CF8118C26C53E67F759100855494D6
:100CDA00855595759104854E56854F57D26043E6E2
:100CEA0080D2AFE52D54066008206A020533020D52
:100CFA000B306C0D206B0A206507158115810215D2
:100D0A00992278003064053065027801E53775F07C
:100D1A0007A4F9E5F028F5F0E9A2F013A2F113A26D
:100D2A00F213F537C394785003753778C3E53795CE
:100D3A00384008D266C295C294C293306002A14577
:100D4A00855056855157D26043E68022207D11C2D4
:100D5A00AF754302D291C292D2AF759F11020F2D85
:100D6A00C2AF754302D291C290D2AF759F11020FE2
:100D7A002D307245207D22C2AF75430390017675EE
:100D8A007E02C293D290D292306204D294A19BC2C4
:100D9A0091D2AF759F01020F2DC2AF754303900127
:100DAA0076757E02C295D292306204D294A1BBC2F9
:100DBA0091D2AF759F21020F2D207D17C2AF7543C7
:100DCA0003900151C293306202D294D2AF759F014F
:100DDA00020F2DC2AF754303900151C295306202D2
:100DEA00D294D2AF759F21020F2D207D11C2AF750B
:100DFA004304D292C290D2AF759F21020F2DC2AF87
:100E0A00754304D290D292C292D2AF759F01020F5B
:100E1A002D307243207D20C2AF7543059001657560
:100E2A007E04C294D291306204D295C139C292D260
:100E3A00AF759F11020F2DC2AF75430590018775DB
:100E4A007E01C294D291306204D293C159C290D227
:100E5A00AF759F11020F2D207D17C2AF7543059004
:100E6A000147C294306202D295D2AF759F11020F28
:100E7A002DC2AF75430590015BC2943062EBD293E9
:100E8A00D2AF759F11020F2D207D13C2AF75430695
:100E9A00D290D292C291D2AF759F01020F2DC2AFEA
:100EAA00754306D292C291D2AF759F21020F2D309F
:100EBA007244207D20C2AF754301900187757E017F
:100ECA00C295D292306204D293C1D7C290D2AF7582
:100EDA009F21020F2DC2AF754301900165757E04F3
:100EEA00C293D290D292306204D295C1F9C292D200
:100EFA00AF759F01E12D207D16C2AF7543019001A8
:100F0A005BC295306202D293D2AF759F21E12DC2A6
:100F1A00AF754301900147C293306202D295D2AFB6
:100F2A00759F01C26622900145757E00C295C294E2
:100F3A00C293D292D291D290C26222788076FF086E
:100F4A0076FF0876FF0876FF0876030876040876A7
:100F5A000A087603087601087601788C7601087605
:100F6A00FF0876FF0876FF0876FF0876FF08760303
:100F7A000876FF0876FF0876FF0876250876D008F7
:100F8A0076FA0876FA0876040876FF087601087673
:100F9A000008767A0876FF08760108760108760056
:100FAA00087603227887E6FFC272BF0302D27278FC
:100FBA0088E6C394036008C27DE630E102D27DC2AE
:100FCA007E7889E630E102D27EC3EF94026008752A
:100FDA008E01D273020FE6758E00C273227880E604
:100FEA00149000809378A4F67881E6149000809398
:100FFA0078A5F67886E61490008D9378A6F6789C04
:10100A00E67538FF75390CB402067538A075390AC9
:10101A00B4030675388275390578A3E61490009AE8
:10102A0093F569120F3022227896E6FA7897E6FB52
:10103A007888E6B40305C3EB940EFB307F047A008C
:10104A007BFFC3EB9AFCC3948250027C82757500C5
:10105A000575EC8575F0A4C3E5F0947D40F222D2C3
:0F106A007F11321205FE7A007B007C101205F414
:10107900E55F2AFA74003BFBDCF37C04C3EB13FB4A
:10108900EA13FADCF7FEC27F113222E5EF20E6030C
:101099007520000520903FFFE520146006901FFF92
:1010A9001460009304600375EF1253D9BF7581C0B2
:1010B90043FF801205EF75EF0243B203E5B3240441
:1010C90020E70DF521E5E320E0068521B343E3019F
:1010D900120F307580FF75A40075F19075D47F7576
:1010E900908775A5BF75F2BF75D50075A60175E224
:1010F90041E4F8F6D8FD756B01120F451215E47835
:10110900988676753001C2AF1206081206181205C4
:10111900FE12061F1205FE1206261205FE1216FD04
:10112900120608120608120603C2AF78FA79FA30D5
:101139008707D9FBD8F7021C00120FAE120FE7116F
:1011490031113278988676120F3075B68075A900FC
:10115900757D0075885075891275C8247591047557
:10116900D84075A82275B80275E690759B80759D63
:101179000075D10E75BC5875BB0675BA1175E88036
:101189001205EFD2AF1208A853DACF207E0343DA53
:1011990020307E0343DA1043DA01C2D8C271120645
:1011A90008D2617B037A0CE55E70077A0CDB0302D7
:1011B90011321205FE207003021132C270E55FC3BD
:1011C900940240E1E52F541F856160F561B560D552
:1011D900DAD5C26153DACF207E0343DA20307E03A9
:1011E90043DA10C2D8C27178A2E67008D274E52F2A
:1011F90054E0F52FC275752900120603307409C32E
:10120900E529940A4002D2751205F4780230740275
:101219007800C3E55F9840F0C2AF120618120618AD
:10122900120618D2AF120608754D007888E6B40385
:101239000261121205F4788CE6C39401500302137B
:1012490012E530C394015003021312207435C3E52B
:101259005F94FF5003021312C2AF12062DD2AF12D0
:101269000603C3E55F940150EFC2AF1206181205D9
:10127900F9120618D2AF120603C3E55F94FF40E9DD
:101289000217827F05D27F1132120603C2AFC27FD5
:101299001132AE5FC3E55F947FD2AF40761205EF9E
:1012A900C2AF12062DD2AFDFDC1169C3EE94057807
:1012B90097F61206081216261217057F0AD27F1111
:1012C90032120603C2AFC27F1132AE5FC3E55F942B
:1012D9007FD2AF50E61205EFC2AF1206181205F918
:1012E900120618D2AFDFD61169EE24057896F612E8
:1012F90006081216261217341206031132C3E55FC7
:1013090094FF50024154021782C3E55F954D400393
:10131900855F4D12060378017988E7B403027805E1
:10132900C3E55F9840024134C2AF12062D12062D63
:1013390012062DD2AF120608753000E4F531F532E8
:101349000531E531F470390532789AE67819146077
:1013590012783214600D787D14600878FA146003ED
:10136900753200C3E53298401715327531B4789952
:101379008676C2AF12062DD2AF789886761206030A
:101389001205F9E52A7005307402213278012074BA
:10139900027806C3E55F9840A77888E6C39403609E
:1013A90003120603E52A7003021132C2AF120F308D
:1013B900E4F522F523F524F525F526F56AD2AF786B
:1013C90085E6C333F568E4F545F546F547F548F58F
:1013D90049F573F52CF52DF53775730875BB1012A2
:1013E90005EF1208ACE5E820ECFBA8BDA9BEE97041
:1013F90001F888741208B075730875BB107887E610
:10140900FE7602120FAE7887EEF6C2AF7564FF1250
:101419000928852264852265852266D2AF75220155
:1014290075240175250175260185636C756D017536
:10143900B69075A903757D017888E6B40307C27D66
:10144900307602D27DD268D269753300120E9212BB
:101459000EB912094812094F12094812094F120907
:0E1469004802147AC2AF120FAED2AF757300F4
:1014770075BB06120BE11206F8120D0C120D56126F
:10148700094F120BD0306D031206F92067031208BB
:101497004B306703120892120D0C120D7B12094F85
:1014A700120BE1306D03120735120D0C120DF412F9
:1014B700094F120BD0306D03120793120D0C120E49
:1014C7001B12094F120BE1306D031207F0120D0CBE
:1014D700120E9212094F1208AC120BD0120D0C12F9
:1014E7000EB91208B012094F306932206B2F856789
:1014F7006485676585636C756D0179187A0CC3E53A
:101507003399400CC269D26A8A357564FF02152483
:10151700C3E55F9401400302147A0215A1306A1BE8
:10152700206B18E535147004C26A816DF535C3E583
:101537005F9401400302147A0215A1753600C3E5D2
:10154700627882985054307404E52A604D7888E6B2
:10155700B40317207D05207607A171307602A171AB
:10156700206B07D26B85676481B978F0306B05858E
:1015770067647820C3E541985002817A306B1BC2BB
:101587006BC27D307602D27DD26A7535128567646B
:10159700817A0536E55F6002A1A4753600C2AF12F5
:1015A7000F307887E6FE7602120FAE7887EEF6E404
:1015B700F522F523F524F525F526F568C26875B6F5
:1015C7008075A900757D00D2AF1205EF120F30307C
:1015D7007409C3E5369405400221326144901A0D1F
:1015E7007820121668E520B45A0CA3121668E52075
:1015F700B4A503021606120F4512162602162590E9
:101607001A0378807B0A121668A308DBF9901A0F71
:10161700788C7B18121668A308DBF9901A2722C268
:10162700AF1216A7121681901A00740E12166DA328
:10163700740412166DA3741412166D901A03788031
:101647007B0A12166CA308DBF9901A0F788C7B18AB
:1016570012166CA308DBF91216BA121698901A27FD
:1016670022E493F622E6438F01538FFD75EF02754F
:10167700B7A575B7F1F0538FFE22438F02438F0151
:1016870075EF0275B7A575B7F1901A0DF0538FFC7A
:1016970022901A0D745AD16D901A0E74A5D16D222D
:1016A7007A3079D07820901A40D168E520F709A3DD
:1016B700DAF7227A3079D0901A40E7D16D09A3DAA8
:1016C700F922AB77A878BB01027984BB020279853E
:1016D700BB03027986BB04027992BB05027987BBFB
:1016E700060279A3BB0702799CBB08027988BB096C
:1016F700027989E8F7227C05120608DCFB22C2AFD3
:1017070012061812061F12062612062D1205F912C6
:10171700061812061F12062612062D1205F91206C2
:101727001812061F12062612062DD2AF22C2AF12BA
:10173700062D12062612061F1206181205F91206A2
:101747002D12062612061F1206181205F912062D6B
:1017570012062612061F120618D2AF22AE77AF78EE
:10176700C2AF1206181206181206181205F9DEF291
:1017770012062D1205F9DFF8D2AF22F105D1FDD1FE
:10178700FD757701757801757900F1637C05AD5FAB
:10179700120608C3ED955F70F5C3E55F9401400A33
:1017A700C3E55F94FF40320217BED1C9D126F105C8
:1017B700C2AF75EF12D1FDDCD50579C3E579940386
:1017C700500280C6D1FD0578E5771490009F93F805
:1017D70008C3E57898500280AED1FDD1FD0577C3E7
:1017E700E577940A5002809C120F45D126C2AF7547
:0417F700EF12D1FD1F
:0319FD0002109441
:101A00000E0414FFFFFFFF03040A0301015AA5019E
:101A1000FFFFFFFFFF03FFFFFF25D0FAFA04FF01DE
:081A2000007AFF01010003FF41
:101A4000234F76736B794D5232304150726F2320A1
:101A500023424C48454C492346333930232020202B
:101A60002020202020202020202020202020202076
:101C0000C2AFC2D353D9BF7581C043B20343FF8073
:101C1000752438752503B1C975EF0275E24043F1AB
:101C20008053A47F75D400D2877DFA780379E67C4F
:101C300010752200752300901DD67B0675249875BB
:101C400025013087028142208708D8FBD9F9DCF7CB
:101C500081B4308708D8FBD9F9DCF781B4B189E4C5
:101C600093A3C39A6004DDC381B4DBDBB17B600264
:101C7000812B7B08E493FAA3B15CDBF87A30B15C8A
:101C8000752200752300B17BEAFCEBFDC3ED94FEE9
:101C9000400EB17B8A278B28ED30E0048A828B834B
:101CA000B17B7AC270D8C3ED94FE601350CEBD00F4
:101CB00025EC60097520007521FF0200008100A855
:101CC00027A9280809D804D90281D3B17FEA89AAB3
:101CD000F281C50D81A0C3ED94035049EDA2E092BD
:101CE000007AC5C3E5829400E583941C50902000DF
:101CF00010438F02438F0175B7A575B7F1F030001F
:101D00001FA827A9280809438F01538FFDD804D99C
:101D100002A12089AAE275B7A575B7F1F0A3A10DBC
:101D2000538FFC817C7AC1BD030CE493A3FAB140CC
:101D3000DCF8B138817C817EAA22AB23B15CEBFA5E
:101D4000EA6222752608C3E52313F523E52213F57D
:101D50002250066323A0632201D526EAB1C9B1C986
:101D600075260AEAF4200102D287300102C287B147
:101D7000C9C3134002C201D526EB22B17FEAFB2082
:101D80008702A17F308702A184752608AE24AF2583
:101D9000C3EF13FFEE13FEB1CDB1C9C3EA13308711
:101DA000024480FA30E703632201C3E52313F523DD
:101DB000E52213F52250066323A0632201D526D91C
:101DC000E52265236523F52222AE24AF250E0FDE22
:101DD000FEDFFCD20122424C48656C693437316326
:041DE000F390060175
:00000001FF
